:03000000020030CB
:100030007590FFD290D291D292D293C280C2801199
:10004000D4311A9001653124311F90017631243169
:100050004F314F314F309014C280C280311F900118
:10006000983124314F314F314F02006C309114C21E
:1000700080C280311F9001A93124314F314F314F5F
:10008000020083309214C280C280311F9001BA31C5
:1000900024314F314F314F02009A309314C280C245
:1000A00080311F9001CB3124314F314F314F02004D
:1000B000B12090A120919E20929B209398D280D233
:1000C00080311F9001DC3124314F314F314F02001C
:1000D0005502003FC285C286C28775A00075A00088
:1000E000743811F9315C740E11F9315C740111F935
:1000F000315C740611F9315C22F5A0C285C286D24A
:1001000087315CC28722F5A0D285C286D287315C56
:10011000C28722740111F9315C22748011F92274B2
:10012000C011F922E49360053106A380F722E4931D
:10013000600AF5993099FDA3C29980F22275A0005A
:10014000758000758920758DE8759850D28E227D56
:10015000067CFF7BFFDBFEDCFADDF6227E327FF9D8
:10016000DFFEDEFA22554E44455247524F554E446B
:100170002043424C4500204641554C5420444554B0
:100180004543544F5220005155414452414E542052
:10019000434F4E54524F4C005749524543555428F3
:1001A00030302D3031294B6D00574952454355545D
:1001B0002830312D3032294B6D0057495245435577
:1001C000542830322D3033294B6D00574952454366
:1001D00055542830332D3034294B6D00414C4C2080
:0D01E000574952455320415245204F4B00D6
:00000001FF
